:020000040800F2
:10000000F81A002001010008511100083D0C0008F9
:100010004D11000829030008C51400080000000065
:10002000000000000000000000000000591300085C
:100030002D03000800000000591200085D1300089D
:100040001B0100081B0100081B0100081B01000820
:100050001B0100081B0100081B0100081B01000810
:100060001B0100081B0100081B0100081B01000800
:100070001B0100081B0100081B0100081B010008F0
:100080001B0100081B0100081B0100081B010008E0
:100090001B0100081B0100081B0100081B010008D0
:1000A0001B0100081B0100081B0100081B010008C0
:1000B0001B0100081B0100081B0100081B010008B0
:1000C0001B0100081B0100081B0100081B010008A0
:1000D0001B0100081B010008A51400081B010008F3
:1000E0001B0100081B0100081B010008DFF80CD0F1
:1000F00000F0E2F800480047A11A0008F81A0020B2
:100100000648804706480047FEE7FEE7FEE7FEE7B1
:10011000FEE7FEE7FEE7FEE7FEE7FEE779140008EC
:10012000ED000008202A04DB203A21FA02F0002129
:10013000704721FA02F3D040C2F1200291400843F7
:100140001946704740EA01039B0703D009E008C93C
:10015000121F08C0042AFAD203E011F8013B00F88C
:10016000013B521EF9D27047D2B201E000F8012BD8
:10017000491EFBD270470022F6E710B513460A4627
:1001800004461946FFF7F0FF204610BD421C10F848
:10019000011B0029FBD1801A704730B480EA0102AC
:1001A00002F0004530F0004221F0004013D090B141
:1001B000C30DD40DC2F31601C0F31600E41A41F4C6
:1001C000000140F400027D34914201D3641C00E040
:1001D0004900002C02DA30BC002070474FF40000C8
:1001E0000023914201D3891A034340084FEA410199
:1001F000F7D151B1914202D14FF0004105E002D256
:100200004FF0010101E06FF0010103EBC4502844FD
:1002100030BC00F019B896230022114600F01DB83A
:1002200020F00040C10DC0F3160040F400007F290B
:1002300001DA00207047962903DCC1F19601C8401D
:1002400070479639884070470029A8BF7047401C06
:10025000490008BF20F00100704710B4B0FA80FCDC
:1002600000FA0CF050EA010404BF10BC704749B119
:10027000CCF1200421FA04F411FA0CF118BF012189
:1002800021430843A3EB0C01CB1D4FEA00614FEA69
:10029000102042BF002010BC704700EBC350104438
:1002A0000029A4BF10BC7047401C490008BF20F0C3
:1002B000010010BC70470000064C074D06E0E068E6
:1002C00040F0010394E8070098471034AC42F6D39D
:1002D000FFF710FF181C0008381C000810B500F0CC
:1002E00085FF0348816A884702494868804710BDF6
:1002F0009C000020E400002010B50A220848018874
:100300000848008800F026FF012805D1044800882D
:100310000449088001F0C4F801F0B0F810BD0000F5
:10032000100000201A00002000BFFEE7704772B6E0
:1003300000BFFEE70021074AD1610749096941F082
:100340000401054A11611146096941F0400111613A
:1003500070470000F8000020002002400021074AFA
:10036000D1610749096941F00201054A116111464D
:100370004861096941F0400111617047F8000020AF
:10038000002002400022054BDA61054A126942F062
:100390000102034B1A61018070470000F800002041
:1003A0000020024000201E49C96801F0100139B147
:1003B0001C49C96941F002011A4AD16140F010009C
:1003C0001749C96801F0040139B11649C96941F0FA
:1003D0000101144AD16140F004001149C96901F0DA
:1003E000010169B10F49C96941F004010D4AD161A8
:1003F00000BF0B49C96921F00101094AD16100BF61
:1004000000BF40F20111884206D10549C96921F0B7
:100410000101034AD16101E00149C86000BF704792
:1004200000200240F800002070B5044600F09CFA5D
:10043000054609E0601C38B124B100F095FA401B74
:10044000A04201D9032070BD1248C06800F001002D
:100450000028EFD10F48C06800F0200020B100BF95
:1004600020200C49C86000BF0A48C06800F0100096
:1004700048B90848C06900F0010020B90548C068C3
:1004800000F0040018B1FFF78DFF0120DBE700202A
:10049000D9E70000002002402DE9F04104460E4655
:1004A0000127002500BF2648007E012802D1022036
:1004B000BDE8F08101202249087600BF20680228AB
:1004C00013D14CF25030FFF7AFFF90BB0120FFF784
:1004D00031FF4CF25030FFF7A7FF0746194800697B
:1004E00020F004001749086123E04CF25030FFF778
:1004F0009BFFF0B94FF0FF303060A56812E028464E
:10050000FFF72CFF4CF25030FFF78EFF07460D48E7
:10051000006920F002000B4908610FB1356007E067
:1005200005F58065D4E9021001EB8020A842E6D8E9
:1005300000BF00BF00200249087600BF3846B7E779
:10054000F8000020002002400348006940F08000CD
:100550000149086100207047002002402DE9FE4F4C
:1005600005468B4617469846012600240020029037
:1005700000BF2448007E012802D10220BDE8FE8F82
:1005800001202049087600BF4CF25030FFF74CFFA5
:10059000064686BB012D02D10120029006E0022D05
:1005A00002D10220029001E00420029000241EE00B
:1005B0002201B946C24648465146FFF7B3FD80B214
:1005C0000190022000FB04B000900199FFF7DAFED1
:1005D0004CF25030FFF728FF06460B48006920F028
:1005E00001000949086106B104E0601CC4B2029828
:1005F0008442DDDB00BF00BF00200249087600BF57
:100600003046BBE7F80000200020024000200849E7
:10061000096901F0800151B10649054A5160064956
:1006200051601146096901F0800101B10120704754
:100630000020024023016745AB89EFCD2DE9F84743
:100640000346002294466EE14FF0010808FA02F4D6
:10065000D1F8008008EA0400A0427DD1DFF8DCA2D6
:10066000D1F80480A8EB0A09D0453AD014DCB8F1DF
:10067000030F50D009DCB8F1000F31D0B8F1010FF1
:100680001CD0B8F1020F49D120E0B8F1110F18D0F9
:10069000B8F1120F42D11EE0B9F5881F25D006DC53
:1006A000B9F5803F20D0B9F5801F37D11AE0B9F5F0
:1006B000001F18D0B9F5041F30D117E0D1F80CC0D5
:1006C0002DE0D1F80C8008F1040C28E0D1F80C8062
:1006D00008F1080C23E0D1F80C8008F10C0C1EE0A6
:1006E00000BF00BF00BF00BF00BF00BFD1F808803F
:1006F000B8F1000F02D14FF0040C0BE0D1F80880E4
:10070000B8F1010F03D14FF0080C1C6102E04FF06B
:10071000080C5C6103E04FF0000C00E000BF00BF7C
:10072000FF2801D8984601E003F104084646FF2857
:1007300002D84FEA820803E0A2F108084FEA8808CD
:100740004746D6F800804FF00F0909FA07F928EA62
:1007500009080CFA07F900E088E048EA0908C6F839
:100760000080D1F8048008F08058B8F1805F7DD116
:1007700000BFDFF8CC81D8F8188048F00108DFF816
:10078000C091C9F81880C846D8F8188008F0010848
:10079000CDF8008000BF00BF4FEAB9384FEA920998
:1007A00058F829504FEA82784FEA18794FF00F082D
:1007B00008FA09F825EA0805DFF88881434502D1DF
:1007C0004FF0000816E0DFF88081434502D14FF07A
:1007D00001080FE0DFF87481434502D14FF00208B1
:1007E00008E0DFF86C81434502D14FF0030801E0D7
:1007F0004FF004084FEA82794FEA197908FA09F8AC
:1008000048EA0505DFF84C814FEA920948F829507B
:10081000D1F8048008F48018B8F5801F0AD1DFF8F9
:100820003881D8F8008048EA0008DFF82C91C9F830
:10083000008009E0DFF82081D8F8008028EA00086D
:10084000DFF81491C9F80080D1F8048008F400188A
:10085000B8F5001F10D1DFF8008108F10408D8F8BE
:10086000008048EA0008DFF8F09000E05AE009F163
:100870000409C9F800800DE0DFF8DC8008F1040805
:10088000D8F8008028EA0008DFF8CC9009F10409C4
:10089000C9F80080D1F8048008F40038B8F5003FAA
:1008A0000ED1DFF8B480A8F10408D8F8008048EA37
:1008B0000008DFF8A490A9F10409C9F800800DE050
:1008C000DFF89480A8F10408D8F8008028EA00082E
:1008D000DFF88490A9F10409C9F80080D1F80480F8
:1008E00008F48038B8F5803F0ED1DFF86C80A8F1AD
:1008F0000808D8F8008048EA0008DFF85C90A9F101
:100900000809C9F800800DE0DFF84C80A8F108085C
:10091000D8F8008028EA0008DFF83C90A9F108091F
:10092000C9F80080521CD1F8008028FA02F8B8F10A
:10093000000F7FF489AEBDE8F887000000001110B9
:100940000010024000080140000C0140001001406E
:100950000014014008000140080401400AB101618F
:1009600001E00B0403617047014800687047000014
:100970000000002003480068034909780844014941
:1009800008607047000000200800002010B50848EB
:10099000006840F0100006490860032000F098F855
:1009A0000F2000F007F800F02BF8002010BD000029
:1009B0000020024070B504460E4800784FF47A716A
:1009C000B1FBF0F00C490968B1FBF0F5284600F0E6
:1009D0001BF908B1012070BD102C07D2002221465E
:1009E000501E00F037F80548046001E00120F2E7EE
:1009F0000020F0E7080000200C0000200400002088
:100A000008B500BF1148806940F001000F498861B6
:100A10000846806900F00100009000BF00BF00BFE1
:100A20000846C06940F08050C8610846C06900F0BF
:100A30008050009000BF00BF00BF0549486820F00B
:100A4000E06040F00070486000BF08BD0010024048
:100A5000000001402DE9F05F80460D461646002754
:100A600000F032FD074639462A46334601F00700BA
:100A7000C0F1070ABAF1040F02D94FF0040A01E0ED
:100A8000C0F1070AD14600F1040ABAF1070F02D2F9
:100A90004FF0000A01E0A0F1030AD4464FF0010A2A
:100AA0000AFA09FAAAF1010A0AEA020A0AFA0CFA8F
:100AB0004FF0010B0BFA0CFBABF1010B0BEA030B34
:100AC0004AEA0B042146404600F006FDBDE8F09FCF
:100AD00000BF00F00702064B19684FF6FF031940EC
:100AE000044B0B4343EA0221014B196000BF7047DE
:100AF0000CED00E00000FA0510B5FFF735FF0446E5
:100B00003D48006840F001003B49086006E0FFF7FF
:100B10002BFF001B022801D9032010BD36480068B6
:100B200000F002000028F2D03348006820F0F800FE
:100B300040F0800030490860FFF716FF04460020AF
:100B40002D49486008E0FFF70FFF001B41F2883194
:100B5000884201D90320E0E72748406800F00C00F4
:100B60000028F0D125482649086026480068FFF78C
:100B700021FF08B10120D0E7FFF7F6FE04461E482A
:100B8000006820F080701C49086006E0FFF7ECFE6A
:100B9000001B022801D90320BFE71748006800F0B6
:100BA00000700028F2D114494860FFF7DDFE0446CA
:100BB0001148006820F410200F49086006E0FFF794
:100BC000D3FE001B642801D90320A6E70A48006869
:100BD00000F400300028F2D10748006820F480209B
:100BE000054908600846406A40F08070486200206D
:100BF000886000BF91E700000010024000127A00F8
:100C00000C0000200400002070B504462546681E34
:100C1000B0F1807F01D301200FE0681E4FF0E0218A
:100C200048610F214FF0FF3000F056FC00204FF0DC
:100C3000E021886107200861002070BD00BFFEE749
:100C40002DE9F04102460B461868C0F30F2595FACE
:100C5000A5F0B0FA80F480E00120A04028400028F0
:100C60007AD0082C04D240F2011000FA04F106E018
:100C7000A4F108004FF00116864046F080615868E4
:100C800008280ED11869D66826EA11260F0A97FAA5
:100C9000A7F7B7FA87F700FA07F73E43D66000BF19
:100CA00000BF586802EB116691FAA1FCBCFA8CFCFB
:100CB0004FEA8C084FF00F0C0CFA08FC376827EA53
:100CC0000C0791FAA1FCBCFA8CFC4FEA8C0C00FAE0
:100CD0000CFC47EA0C07376000BF5868012802D0B7
:100CE0005868092838D1986802EB116691FAA1FC7E
:100CF000BCFA8CFC4FEA8C084FF0030C0CFA08FC91
:100D0000376827EA0C0791FAA1FCBCFA8CFC4FEA81
:100D10008C0C00FA0CFC47EA0C07376000BFD8685F
:100D200002EB116691FAA1FCBCFA8CFC4FEA8C082C
:100D30004FF0040C0CFA08FC376827EA0C0791FA0C
:100D4000A1FCBCFA8CFC4FEA8C0C00FA0CFC47EAC4
:100D50000C07376000BF00BF641C25FA04F00028B0
:100D60007FF47AAFBDE8F08110B5044600F0AAFA2E
:100D70002060206800F072FA6060606800F07EFA1F
:100D8000A060606800F08CFAE06010BD0149086066
:100D9000704700000C0000202DE9FF4104460D467D
:100DA00001270026204600F046F8002833D1E968E4
:100DB0006868084329690843E16841F20C6291437D
:100DC0000843E060A868216921F440510143216192
:100DD00000BF6869616921F440710143616100BF2E
:100DE0006846FFF7C1FF0E48844201D1039E08E028
:100DF0000C48844201D1029E03E00B48844200D19A
:100E0000029E46B1286830B10027314620462A6844
:100E100000F016F800BF384604B0BDE8F0810000CD
:100E20000038014000440040004800400146086886
:100E3000C0F3401070470146C868C0F340307047A7
:100E400070B501EBC10303EB01139400B3FBF4F3A2
:100E500001EBC10404EB01149500B4FBF5F4642527
:100E6000B4FBF5F404EBC40505EB0414A3EB840315
:100E7000322404EB03136424B3FBF4F303F0F00314
:100E800001EBC10404EB01149500B4FBF5F46425F7
:100E9000B4FBF5F403EB041401EBC10303EB011302
:100EA0009500B3FBF5F301EBC10505EB01159600C9
:100EB000B5FBF6F56426B5FBF6F505EBC50606EBC6
:100EC0000515A3EB8503322505EB03136425B3FB5E
:100ED000F5F303F00F0323449BB2836070BD000061
:100EE00000B585B00020019002900390049000BFEF
:100EF0003548806940F020003349886108468069A0
:100F000000F02000009000BF00BF00BF08468069CD
:100F100040F0040088610846806900F004000090F9
:100F200000BF00BF00BF0846806940F0080088612C
:100F30000846806900F00800009000BF00BF002252
:100F400041F612012148FFF709FD012241F2030198
:100F50001F48FFF703FD00224FF4F0711C48FFF714
:100F6000FDFC41F612000190012002900020039048
:100F70000220049001A91548FFF760FB41F2E3004D
:100F8000019001200290002003900320049001A909
:100F90000F48FFF753FB4FF480700190012002903F
:100FA000002003900220049001A90948FFF746FBA6
:100FB0004FF40070019000200290039001A90448B2
:100FC000FFF73CFB05B000BD0010024000080140E7
:100FD000000C01402DE9F0418EB01C2107A8FFF75D
:100FE000CAF8142102A8FFF7C6F84FF4003052499E
:100FF000C9690143504AD1611146C9690140019153
:1010000000BF00BF04201146896901439161114668
:1010100089690140019100BF00BF40F20440029085
:1010200009200390032004900020059002A9434862
:10103000FFF706FE40F6080002900420039002A984
:101040003E48FFF7FDFD26213D4B1B68C3F3022000
:10105000002425460346C3F1070CBCF1040F02D956
:101060004FF0040C01E0C3F1070C674603F1040CD8
:10107000BCF1070F02D24FF0000C01E0A3F1030C0A
:1010800066464FF0010C0CFA07FCACF1010C0CEABF
:10109000040C0CFA06FC4FF0010808FA06F8A8F157
:1010A000010808EA05084CEA080200BF002904DB31
:1010B0001007030E2348435407E01007040E20488E
:1010C0000C3001F00F031B1FC45400BF2620002862
:1010D00009DB00F01F02012191404209920002F158
:1010E000E022C2F8001100BF4FF416500790002014
:1010F000089009900A900C200B9000200C900D9005
:1011000007A91148FFF748FE00BF0F48006920F407
:1011100090400D4908610846406920F02A00486166
:1011200000BF00BF0846C06840F40050C86000BF60
:101130000EB0BDE8F0810000001002400008014040
:101140000CED00E000E400E00044004000BFFEE7DA
:1011500000BFFEE710B503461446E01882B29A427B
:1011600005DD914201DA994207DA012010BD914272
:1011700003DB994201DA0120F8E70020F6E70000DE
:10118000154909880144144A118014490988014409
:10119000124A1180124909880144114A11800F49ED
:1011A0000988B1F57A7F07D300210C4A11800D49D7
:1011B0000988491C0B4A11800949098842F21072BA
:1011C000914207D30021064A118007490988491C2A
:1011D000054A118070470000100000201600002012
:1011E00018000020120000201400002000201049E8
:1011F0000880104908801049088010490880084676
:1012000000880F4908800D4800880E4908800B4867
:1012100000880D490880094800880C490880074863
:1012200000880B490880054800880A4908807047F3
:1012300016000020180000201200002010000020DE
:101240001A0000201C0000201E00002020000020AA
:10125000220000202400002070470000014600BF4B
:101260000448406800F0F0000009034A125C21FACB
:1012700002F0704700100240E41B0008014600BF66
:101280000548406800F4E060044A02EB1020027850
:1012900021FA02F07047000000100240F41B000821
:1012A000014600BF0548406800F46050044A02EB64
:1012B000D020027821FA02F07047000000100240AE
:1012C000F41B000810B5002400BF0B48406800F074
:1012D0000C0020B1042804D0082808D103E0074CF2
:1012E00007E0064C05E000F00BF8044601E0034C73
:1012F00000BF00BF204610BD0010024000127A005F
:101300000021002200BF1148406800F480300246EE
:101310001AB1B2F5803F0CD101E00D490BE000BFDE
:101320000A484068C0F34040401C0A4BB3FBF0F150
:1013300001E0074900BF00BF00BF0448406800F457
:101340007010022303EB90404843704700100240A6
:1013500000093D0000127A007047000010B501201E
:10136000FFF70EFF05480121826B904704480121D9
:10137000826B9047FFF7FEFA10BD00005800002076
:101380009C00002010B502203849096821F00701AF
:101390000143364A116000BF00BF00BF33480068F8
:1013A00000F007000228F8D100BF3148006840F47F
:1013B00080302F49086000BF00BF00BF2C48006884
:1013C000C0F340400028F8D04FF480304FF4E011D3
:1013D000274A526822F47C1200F440330B431A432C
:1013E000234B5A6000BF00BF1846006840F0807071
:1013F0001946086000BF00BF00BF1D480068C0F369
:1014000040600028F8D000201949496821F0F00117
:101410000143174A516000BF10151146496821F475
:10142000E0610143516000BF00201146496821F48A
:1014300060510143516000BF02201146496821F00C
:1014400003010143516000BF00BF00BF084840686E
:1014500000F00C000828F8D10648FFF797FC0F2091
:10146000FFF7A8FA08B1FEF762FF10BD00200240A6
:101470000010024000A24A047047000010B5054861
:10148000016C88470448016C884704498868804794
:1014900010BD0000580000209C000020E400002047
:1014A0007047000010B50548FFF7C0FC28B100BF29
:1014B000024800680248416B884710BD0044004064
:1014C0009C00002000BFFEE702480068C0F3022035
:1014D000704700000CED00E010B5002804DB0A079F
:1014E000130E054A135406E00A07140E034A00F0CF
:1014F0000F031B1FD45410BD00E400E018ED00E002
:1015000002E008C8121F08C1002AFAD170477047CC
:10151000002001E001C1121F002AFBD1704700002A
:1015200070B5144C144920680840B0F1005F1FD119
:1015300072B6FFF7E1FA00204FF0E0210861486140
:10154000886100BF09E04FF0FF320C4941F82020CC
:101550000B4941F82020411CC8B20828F3DB65681C
:10156000206880F3088800BF62B6A84700BFFEE786
:1015700070BD0000002800080000FE2F80E100E0A0
:1015800080E200E010B586B0044600200190029091
:1015900004940120059001A902A8FEF77DFF06B082
:1015A00010BD10B50021C163416801B910BD41688B
:1015B00000BF00BF00BF01F10C0353E8003F43F040
:1015C000200201F10C0343E80024002CF3D100BFFA
:1015D00000BF00BFEAE738B5044660684168C9B299
:1015E00000916946206800F0C2FA204600F03CF8FD
:1015F00038BD000070B50446A08C618C884227DAA3
:10160000206880892084204600F034F8208CE18B0B
:1016100088421DDC208CD8B1208C40F24C4188429D
:1016200003DD206800F057FA12E0002506E0094AC1
:101630005119206800F057FA681C85B2208CA84226
:10164000F5DCE06B20B1218C22460248E36B984721
:1016500070BD0000B009002090F82620012A02D1B8
:10166000428C0A4442847047012180F826100021F0
:1016700041847047002180F826104184704730B5BE
:101680000B4600210CE000BF44682568C5F3C01577
:10169000002DF9D05D5C4468656000BF4C1CA1B2B0
:1016A0009142F0DB30BD0121817470470020034975
:1016B0000968087002480349C8637047F0000020B9
:1016C000C91600089C0000202DE9F74F88B0064697
:1016D0000F46002007900690AF4800680078022867
:1016E00002D10BB0BDE8F08F30785A2801D1042F19
:1016F00000DAF6E7B078717840EA0129381F4845EA
:1017000002D0032006900BE0781E81B2304600F034
:1017100059FA8246781E315C514501D0012006906D
:101720009E490A980860F478351D072C6FD2DFE8CF
:1017300004F06E042D6FA9E7C800012096490968DE
:1017400008709748FEF722FD401C00F0FF08424653
:1017500093499448FEF7F6FCC346A5209149C91E5B
:1017600008700BF1010048708C7008464078811CAD
:101770008C48C01E00F026FA8A4AD21E0BF10301E3
:10178000505410464078C01C0790D7E068782978FC
:1017900040EA01200590E878A97840EA012B7E48CC
:1017A0000068A0F802B05846FEF735FD01460190EA
:1017B0004FF08940FEF7F1FC03900598FEF72BFDF2
:1017C00002900399FEF7E9FC0490FEF729FD80B230
:1017D0000590059800F048F94FF00008A5207149E0
:1017E000C91E087008F1010048708C7008464078E6
:1017F000811C6C48C01E00F0E5F96A4AD21E08F14F
:101800000301505410464078C01C079096E092E0C7
:101810006878297840EA0128A9F1030080B2059090
:101820005D480068408800FB08F00490A81C039005
:101830005D4A04998818059A039900F0EDF84FEA7B
:1018400028205849C91EC870084680F804804FF007
:10185000020BA52101700BF101005249C91E48700D
:101860008C7008464078811C4E48C01E00F0AAF9D2
:101870004C4AD21E0BF10301505410464078C01C54
:1018800007905BE04FF000080220434909680870A8
:10189000A5204449C91E087008F1010048708C70E9
:1018A00008464078811C3F48C01E00F08BF93D4A35
:1018B000D21E08F10301505410464078C01C079016
:1018C0003CE04FF0020828783649C91EC870687895
:1018D0000871A520087008F1010048708C70084656
:1018E0004078811C2F48C01E00F06CF92D4AD21E92
:1018F00008F10301505410464078C01C07901DE0C9
:101900004FF00008A5202749C91E087008F1010002
:1019100048708C7008464078811C2248C01E00F038
:1019200051F9204AD21E08F1030150541046407864
:10193000C01C079002E00220069000BF00BF06987E
:1019400030B101280AD0022809D003281FD107E0AE
:101950001448C01E079900F029F819E000BF00BF25
:10196000A5201049C91E0870012048708C70069887
:10197000C87004210B48C01E00F024F90949C91E93
:10198000087105210748C01E00F010F800E000BFF4
:1019900000BF00BFA5E60000F0000020F40000201A
:1019A000031C0008D71600200028000870B5044664
:1019B0000D460648006838B1044800682A462146AA
:1019C000C36A02480068984770BD0000F400002018
:1019D00010B50E480068007820B101280FD0022809
:1019E00011D10DE04FF47A72094801880948008846
:1019F000FFF7B0FB012801D1FFF792FD04E003E0FF
:101A0000FFF78EFD00E000BF00BF10BDF00000201A
:101A100010000020E00000202DE9F04180460D4636
:101A20001746FEF7F3FD00BF30200E49C86000BF27
:101A3000002411E0601CB84204DA295D285C41EA08
:101A4000002600E02E5D08EB040132460023012051
:101A5000FEF784FDA01C84B2BC42EBDBFEF774FDF4
:101A6000BDE8F0810020024070B50546FEF7CEFDCE
:101A700000BF30200849C86000BF002406E00749C5
:101A800001EB8420FFF77EFD601C84B2AC42F6DBE4
:101A9000FEF75AFD70BD000000200240002800083B
:101AA000FEF774FFFFF76EFCFFF71AFAFFF792FAE2
:101AB000FEF714FC01E0FEF71FFCFCE770B50346DF
:101AC0000C4603E014F8015B03F8015B151EA2F15C
:101AD0000102F7D170BD00B9704700214161016179
:101AE000C16000BFF8E770B504460D460CB9002090
:101AF00070BDE06808B90020FAE745B1D4E90006F6
:101B0000236903FB060132462846FFF7D7FF206909
:101B1000401CA16890FBF1F201FB12002061E0681B
:101B2000401EE0600120E3E770B504460D460CB9A5
:101B3000002070BDD4E90210884201D10020F8E7EE
:101B400045B1D4E90016636903FB06103246294605
:101B5000FFF7B4FF6069401CA16890FBF1F201FB44
:101B600012006061E068401CE0600120E1E770B5B0
:101B700004460D460CB9002070BDD4E9021088421D
:101B800004DA29462046FFF7CFFFF5E745B1D4E94F
:101B90000016636903FB061032462946FFF78EFFE5
:101BA0006069401CA16890FBF1F201FB12006061CA
:101BB0002069401CA16890FBF1F201FB120020613A
:101BC0000120D9E710B502460B460024002104E0AD
:101BD000505C2044C4B2481C81B29942F8DB604298
:101BE000C0B210BD000000000000000001020304AC
:101BF000060708090000000001020304081C304425
:101C0000586C8056302E3030312E300000000000ED
:101C10000000000000000000381C00080000002048
:101C2000F800000000150008301D0008F800002032
:101C3000001A00001015000800000000100000004D
:101C40000100000000127A00000000000000000007
:101C50000000000000000000000000000000000084
:101C600018010020010000004C04000000000000EA
:101C700000000000000000006405002001000000DA
:101C80004C04000000000000000000000000000004
:101C900028000020003801400000024000000240FF
:101CA00005040100FC0D00201C0E002020004C0447
:101CB000000000000A000000A31500087F160008BD
:101CC000A7160008D71500085916000800000000E4
:101CD000F5150008400000200044004000000240CC
:101CE000000002400201010068120020881200205A
:101CF00020004C040000000005000000A3150008AF
:101D00007F160008A7160008D71500085916000806
:101D100000000000F51500080000000000000000B1
:101D2000AD160008D1190008E400002000000000F2
:04000005080000ED02
:00000001FF
